:100000000C94E5000C9400130C94D9120C94B212C9
:100010000C948B120C940D010C940D010C94641231
:100020000C940D010C9400140C945B0C0C94CD0CEE
:100030000C940D010C940D010C940D010C940D0108
:100040000C940D010C940D010C940D010C940D01F8
:100050000C940D010C940D010C940D010C941A12CA
:100060000C940D010C94380F0C94120F0C940D018C
:100070000C940D010C940D010C940D010C940D01C8
:100080000C940D010C940D010C940D010C940D01B8
:100090000C94CC030C940D010C940D010C940D01E7
:1000A0000C940D010C94D0010C940D019C0F9F0F2A
:1000B0008E0F920F980FC00FC00FC00FA30FA70F86
:1000C000AB0FB10FB50FC00FBB0F080B0002020240
:1000D00001000904000001020200000524001001D3
:1000E0000524010101042402060524060001070578
:1000F000810310004009040100020A000000070506
:1001000002024000000705830240000004030904C6
:1001100012010002EF02014041233680000101027A
:10012000030141726475696E6F204C4C430041724B
:100130006475696E6F204C656F6E6172646F00004C
:10014000000000240027002A002D003000000000DD
:1001500000250028002B002E0031000000000023A5
:1001600000260029002C002F0004040404040304CA
:100170000502020202040302020202060606060645
:100180000604040202020404040802011040804034
:1001900010204080408008020401804020100201AD
:1001A000108010204040200000000200090F0000D5
:1001B000030401000C00000000000000000000002B
:1001C0000000000000003D226D1B11241FBECFEF78
:1001D000DAE0DEBFCDBF12E0A0E0B1E0E6E2F0E59C
:1001E00002C005900D92A031B107D9F724E0A0E13B
:1001F000B2E001C01D92AC38B207E1F710E0C4EEE6
:10020000D0E004C02197FE010E941125C33ED10712
:10021000C9F70E949C1B0C9406280C94000085EDE5
:100220008093BC008091BC0084FDFCCF1092F6024C
:10023000089540913D02262F30E0240F311D2132D8
:100240003105DCF42091F6022430C9F4FC0180E091
:1002500090E0861758F430913D022191DC01A55EB3
:10026000BD4FA30FB11D2C930196F3CF80913D029A
:10027000680F60933D0280E0089581E0089582E078
:1002800008950895E091AF028091AE02E81730F42E
:10029000F0E0E055FD4F808190E008958FEF9FEFF3
:1002A00008959091AF028091AE02981750F4E92F13
:1002B000F0E0E055FD4F208130E09F5F9093AF026A
:1002C00002C02FEF3FEFC90108958091AE0290E088
:1002D0002091AF02821B91090895CF92DF92EF9295
:1002E000FF920F931F93CF93DF937C01262F972FBD
:1002F0008A018091F702882391F0C62FD72F6E01D3
:10030000C40ED51ECC15DD0571F06991D701ED91B4
:10031000FC910190F081E02DC7010995F3CF642F86
:10032000822F0E941901C801DF91CF911F910F9177
:10033000FF90EF90DF90CF900895CF93DF931F92BF
:10034000CDB7DEB769832091F7022223D1F0209147
:100350001903203240F021E030E0FC013383228396
:1003600080E090E015C08091F802E82FF0E0E750BF
:10037000FD4F998190838F5F8093F80280931903DA
:1003800005C061E0CE0101960E94190181E090E074
:100390000F90DF91CF910895089580E090E0089547
:1003A0001F920F920FB60F9211246F927F928F922D
:1003B0009F92AF92BF92CF92DF92EF92FF920F93F4
:1003C0001F932F933F934F935F936F937F938F93DD
:1003D0009F93AF93BF93CF93DF93EF93FF9380915E
:1003E0009402909195029C0121503109309395021D
:1003F00020939402892B09F0B0C110927200789476
:100400008091C100807F84608093C10083E08093ED
:10041000BF0088EE8093D1001092BF001092D200EE
:1004200081E0809319018091960290919702892B27
:1004300009F493C18091640281118FC190900801E9
:1004400080916302882321F08091620281117BC137
:100450007724739470ECA72E7DE5B72EEAE06E2E1C
:10046000F4E08F2EA0EDCA2EA7E0DA2EB4E0EB2E3A
:10047000F12C04EF11E0CFE0D0E00E945114209164
:100480009602309197022F5F3F4F3093970220934F
:100490009602853609F45EC07CF5813609F49EC06B
:1004A00024F58C3309F452C08E3309F44DC08132E7
:1004B00009F08FC080920801D0920501C09204011A
:1004C000F0920701E09206011093030100930201EC
:1004D000D0930101C0930001109263029090080133
:1004E0008091020190910301C8CF833689F10CF409
:1004F00078C000E022E077C08D36A9F16CF4873631
:1005000079F15CF18C3609F064C00E94721490930A
:100510000701809306014EC08237D1F14CF48F362B
:1005200009F057C00E947214982E80930801A5CF3D
:10053000843789F1863709F04CC00E947214909379
:1005400001018093000199CF939497CF9A9495CF0E
:1005500000E01FC000E024E046C000E025E043C00A
:1005600000E027E040C00E9451148C3619F410922C
:10057000630204C07092630210926202809196023C
:10058000909197020196909397028093960275CF6F
:1005900001E020E028C00E947214BC01C5010E9445
:1005A000E924669EC001679E900D11249093050179
:1005B00080930401809104019091050160910601EE
:1005C000709107010E94E924709303016093020176
:1005D00054CF1092970210929602BFC000E029E01B
:1005E00002C000E02BE0122F3CE0939E100D11247E
:1005F0000E945114982F977F933259F4809196025C
:1006000090919702019690939702809396021F5FB4
:10061000EFCF8D3269F48091960290919702019606
:10062000909397028093960211500E945114F1CF3B
:10063000C0910201D09103018153883058F4C091D8
:100640000401D09105010E947214BC01CE010E94E8
:10065000E924EB017E01F694E7940E9451148E3256
:1006600061F480919602909197020196909397027F
:1006700080939602CE0DDF1DEECFFE0180916302C6
:10068000882349F0CE0196958795809362028091E8
:100690006202E81BF109C0910001D0910101011132
:1006A00004C01F3F11F0C11105C040E0BF0188EE3A
:1006B00093E046C0113130F020EF210F203618F0C2
:1006C0002FE501C020E0822F6CE00E94DD24682F1E
:1006D00074EF7603A0011124BA01620F711D9B0112
:1006E0006C30710540F4220F331FD901A65CBE4F58
:1006F0002D913C9102C020E030E0873081F0082E3F
:1007000002C0220F331F0A94E2F7823028F0C90199
:1007100005966AE070E00CC0C90190580CC0C90190
:1007200026E0880F991F2A95E1F7029665E070E0B0
:100730000E94E924CB014C2FC03108F04FE0BF01EB
:100740000E949A140AC06091620270E040E088EE54
:1007500093E00E949A1410926202FF91EF91DF9150
:10076000CF91BF91AF919F918F917F916F915F9149
:100770004F913F912F911F910F91FF90EF90DF903C
:10078000CF90BF90AF909F908F907F906F900F9081
:100790000FBE0F901F9018951F920F920FB60F92D9
:1007A00011242F933F934F935F936F937F938F9376
:1007B0009F93AF93BF93EF93FF938091B900887F8E
:1007C000803609F49CC068F5883209F45BC090F467
:1007D000803109F454C038F4882309F4F6C0883015
:1007E00009F44DC0F6C0883109F44CC0803209F4D8
:1007F0005DC0EFC0803409F468C048F4803309F468
:1008000055C0883309F0E5C08093F402D8C0803524
:1008100009F44FC0883509F45DC0883409F0D9C0A7
:10082000D6C0883909F4C7C0A8F4883709F467C06E
:1008300038F4883609F463C0803709F460C0C9C051
:10084000883809F4B8C0803909F45FC0803809F0ED
:10085000C0C05BC0803B09F486C038F4803A09F41C
:1008600066C0883A09F47FC0B4C0803C09F4A7C0D0
:10087000883C09F4A4C0883B09F48AC0AAC08091CE
:10088000D10210C09091F3028091F202981770F596
:10089000E091F30281E08E0F8093F302F0E0EE52DC
:1008A000FD4F80818093BB0085EC86C08093F4026D
:1008B0008EC0E091F30281E08E0F8093F30280916D
:1008C000BB00F0E0EE52FD4F80839091F3028091E7
:1008D000F2026EC0E091F30281E08E0F8093F3028A
:1008E0008091BB00F0E0EE52FD4F80838091F502D5
:1008F00081116DC081E08093D00284EA61C083E001
:100900008093F60210926102CFCF80916102803213
:1009100008F051C0E091610281E08E0F8093610286
:100920008091BB00F0E0EF5BFD4F8083BDCF85EC95
:100930008093BC001092F60280916102803230F404
:10094000E0916102F0E0EF5BFD4F10826091610287
:1009500070E0E0913F02F091400281E492E009955D
:100960001092610236C084E08093F60210923E023B
:1009700010923D02E0913B02F0913C02099580917A
:100980003D02811105C081E080933D0210921B025F
:10099000E0913E0281E08E0F80933E02F0E0E55E42
:1009A000FD4F80818093BB0090913E0280913D027B
:1009B000981708F479CF85E88093BC000AC085ECCD
:1009C0008093BC001092F60204C01092F4020E94C0
:1009D0000F01FF91EF91BF91AF919F918F917F9107
:1009E0006F915F914F913F912F910F900FBE0F909C
:1009F0001F90189580911202811105C081E08093AB
:100A000012020E94BB13F89480919A0290919B026B
:100A1000789490931402809313026EE873E00E941E
:100A2000FD247093180260931702809112028111C5
:100A300005C081E0809312020E94BB13F89480915C
:100A400098029091990278949093160280931502DF
:100A50006EE873E00E94FD2470931A0260931902FD
:100A600008958F929F92AF92BF92CF92DF92EF92B2
:100A7000FF920F931F930E949B16E0901704F09033
:100A800018048091700290917102E81AF90AF092AC
:100A90001102E09210020E94151120916E02309115
:100AA0006F02AB01421B530B9A0170936F0260936C
:100AB0006E02D7010E94172520E030E040EE50E0A2
:100AC0000E941E25EDE8AE2EF8E3BF2EACE0CA2E44
:100AD000DD24D394E12CF12C00E010E00E945A2593
:100AE00049015A018091760290917702A091780293
:100AF000B0917902880D991DAA1DBB1D80937602C5
:100B000090937702A0937802B09379029D015527C4
:100B100037FD5095452FA8E6B1E00E94AA23BB27D8
:100B200097FDB095AB2F8093720290937302A093C0
:100B30007402B09375021F910F91FF90EF90DF90B8
:100B4000CF90BF90AF909F908F900895CF93DF93F9
:100B500000D000D000D0CDB7DEB761E0CE01019665
:100B60000E942C1AEEE7F2E0A8E6B2E089819A81B1
:100B70002D913C911197821B930B918380838B81E4
:100B80009C8112962D913C911397821B930B93831A
:100B900082838D819E8114962D913C911597821BA5
:100BA000930B9583848326960FB6F894DEBF0FBE11
:100BB000CDBFDF91CF910895CF92DF92EF92FF9258
:100BC0000F931F93CF93DF93CDB7DEB72C970FB65C
:100BD000F894DEBF0FBECDBF10E080916E041817F1
:100BE00088F4E0916C04F0916D0483E0189FE00DAF
:100BF000F11D112480818F3118F462E00E94AB1046
:100C00001F5FEBCF80916F048F3170F460E00E9422
:100C10007B1061E080916F040E94AB10809177049B
:100C2000909178040E940A1180917004909171044F
:100C3000892B01F58CE0EEE2F1E0DE0111960190E6
:100C40000D928A95E1F76CE070E080E090E00E9400
:100C50002E27009779F02CE0FE013196DC010190FF
:100C60000D922A95E1F7909371048093700486E0C9
:100C70008093720420916C0430916D0480E0909117
:100C80006E04891750F4F90193E0899FE00DF11D7E
:100C90001124128211828F5FF2CF10E080917204D2
:100CA000181708F07EC09091700480917104E92FAC
:100CB000F82FE10FF11DE10FF11DC080D1804091AF
:100CC000730450917404B60180E090E00E948E138A
:100CD00080917504909176040E940A1100E0809141
:100CE0006E040817E0F483E0089F70011124E0917E
:100CF0006C04F0916D04EE0DFF1D80818F3168F45E
:100D00000E945210892B49F4E0916C04F0916D041B
:100D1000EE0DFF1D81818F5F81830F5FE0CF0E9409
:100D2000741380917704909178040E940A11409185
:100D3000730450917404B60181E090E00E948E1318
:100D400080917504909176040E940A1100E08091D0
:100D50006E040817E0F493E0099F70011124E091FC
:100D60006C04F0916D04EE0DFF1D80818F3168F4ED
:100D70000E945210892B49F4E0916C04F0916D04AB
:100D8000EE0DFF1D82818F5F82830F5FE0CF0E9497
:100D9000741380917704909178040E940A111F5F68
:100DA0007DCF84E10E94B31510916E04811758F431
:100DB000E0916C04F0916D0493E0899FE00DF11DCA
:100DC0001124818101C080E08093840286E10E9429
:100DD000B315811758F4E0916C04F0916D0493E021
:100DE000899FE00DF11D1124818101C080E0809375
:100DF000850286E10E94B315811758F4E0916C04D6
:100E0000F0916D0493E0899FE00DF11D1124828122
:100E100001C080E08093860284E00E94B3158117B0
:100E200058F4E0916C04F0916D0493E0899FE00D1B
:100E3000F11D1124828101C080E0809387022C96ED
:100E40000FB6F894DEBF0FBECDBFDF91CF911F91DB
:100E50000F91FF90EF90DF90CF9008950E940E12B7
:100E600020917C0230917D02621B730B70937B0298
:100E700060937A020895882311F0479A01C0479839
:100E80003F9A08958F929F92AF92BF92CF92DF9236
:100E9000EF92FF9280917E0290917F028759910993
:100EA0008D35914008F042C081E00E943B07C09020
:100EB0000901D0900A01E0900B01F0900C01A7010C
:100EC000960160E070E088EC91E40E9425240E9485
:100ED00097244B015C01A701960160E070E084ED6E
:100EE00092E40E9425240E949724DC01CB01B401E6
:100EF0000E9427130E940E1270937D0260937C0261
:100F00000E942E0780917A0290917B02843691058F
:100F100008F085C00E942E070E94A60580918202DB
:100F200090918302893791056CF379C08091820298
:100F300090918302895791098B37914008F042C004
:100F400081E00E943B07C0900901D0900A01E09027
:100F50000B01F0900C01A701960160E070E088ECB5
:100F600092E40E9425240E9497244B015C01A70172
:100F7000960160E070E088ED91E40E9425240E94D3
:100F80009724DC01CB01B4010E9427130E940E12AA
:100F900070937D0260937C020E942E0780917A02FA
:100FA00090917B028436910508F039C00E942E078B
:100FB0000E94A60580917E0290917F02873991055B
:100FC0006CF32DC05D98559AC0900901D0900A012C
:100FD000E0900B01F0900C01A701960160E070E039
:100FE00088EC92E40E9425240E9497244B015C0126
:100FF000A701960160E070E084ED92E40E94252450
:101000000E949724DC01CB01B401FF90EF90DF90A8
:10101000CF90BF90AF909F908F900C942713FF902C
:10102000EF90DF90CF90BF90AF909F908F900895FA
:1010300081E00E943B0781E090E00E949F1A0E949D
:10104000A60580917E0290917F02855F9140833852
:10105000934050F420918002309181022D52314012
:1010600081E02F38314008F080E0209182023091F9
:101070008302255F31402338334008F02AC1209194
:101080008002309181022D5231402F38314008F0DA
:1010900020C1882309F495C00E942C2322E030E06F
:1010A00040E050E00E948B23DC01CB010196A11DA2
:1010B000B11D81309105A105B10509F0B6C16EE6FB
:1010C00070E08AE690E00E9427130E940E1270934F
:1010D0007D0260937C020E942E0780917A0290919B
:1010E0007B028C32914048F40E942E076EE670E03D
:1010F0008AE690E00E942713F0CF0E94A605809117
:101100007E0290917F028639910584F4809182025B
:1011100090918302883791054CF40E94A60564E6FD
:1011200070E08AE690E00E942713E9CF10927602E1
:101130001092770210927802109279021092720245
:101140001092730210927402109275020E9431057F
:101150008091720290917302A0917402B091750215
:101160008A359105A105B1052CF50E9431050E9433
:10117000A6058091820290918302895791098B374D
:10118000914028F464E670E080E090E010C0809127
:101190007E0290917F028759910964E670E08D3557
:1011A000914018F485E390E002C08BE190E00E944A
:1011B0002713CECF64E670E08AE690E00E94271302
:1011C00065C00E942C2322E030E040E050E00E9405
:1011D0008B23613009F07FC0109276021092770263
:1011E0001092780210927902109272021092730299
:1011F0001092740210927502109218021092170247
:101200000E9431058091720290917302A091740244
:10121000B0917502893D9F4FAF4FBF4FACF00E9418
:1012200031050E94FA040E94A60569E170E08AE691
:1012300090E00E94271380917E0290917F0287594F
:1012400091098D359140F0F60E9431050E940E12F1
:1012500070937D0260937C02809172029091730280
:10126000A0917402B09175028C3A9F4FAF4FBF4F5F
:101270006CF00E942E070E9431050E94A605809105
:101280007A0290917B02893B9B4020F080E090E0C5
:101290000C949F1A80917E0290917F028759910948
:1012A0008D35914018F460E070E00EC080918202AC
:1012B00090918302895791098B37914018F462E32A
:1012C00070E002C069E170E08AE690E00E942713B6
:1012D000C3CF81111CC064E670E08AE690E00E94F2
:1012E00027130E940E1270937D0260937C020E946D
:1012F0002E0780917A0290917B02883E934030F6CF
:101300000E942E070E94A6050E944207F2CF0E946B
:101310002C2322E030E040E050E00E948B2361303B
:10132000D1F6109276021092770210927802109203
:10133000790210927202109273021092740210924B
:10134000750210921A02109219020E9431058091C2
:10135000720290917302A0917402B0917502889705
:10136000A105B1055CF40E9431050E94FA0464E60F
:1013700070E08BE190E00E942713E9CF10921A02EF
:10138000109219020E9431058091720290917302AD
:10139000A0917402B091750285359105A105B10542
:1013A0005CF40E9431050E94FA0464E670E08BE16F
:1013B00090E00E942713E8CF64E670E08AE690E0B0
:1013C0000E9427130E940E1270937D0260937C028C
:1013D0000E942E0780917A0290917B02883E934072
:1013E00068F40E942E070E94A605809182029091C7
:1013F0008302895791098B37914060F70E940E1242
:1014000070937D0260937C020E942E0780917A0285
:1014100090917B02883E934008F038CF0E942E07BF
:101420000E94A6050E944207F1CF823009F4D4CE73
:1014300052CF0E94F8274091910250919202209140
:101440008F023091900242175307B4F49091E80054
:101450009570E1F39091E80092FD19C08093F1003E
:10146000809191029091920201968F739927892B16
:1014700019F48EEF8093E80080919102909192028E
:101480000196909392028093910281E0089580E00A
:101490000895DF92EF92FF920F931F93CF93DF9304
:1014A000D82E8A017B01E40EF51EEB01CE15DF0577
:1014B00071F0D7FE03C0FE01849101C088810E94B3
:1014C0001B0A21968111F2CF8FEF9FEF01C0C80157
:1014D000DF91CF911F910F91FF90EF90DF900895D2
:1014E000615030F02091F100FC0120830196F8CF8B
:1014F000289884E680937A040895CF92DF92EF9241
:10150000FF920F931F93CF93DF936C017A018B01AE
:10151000C0E0D0E0CE15DF0589F0D8016D918D01D6
:10152000D601ED91FC910190F081E02DC601099565
:10153000892B11F47E0102C02196ECCFC701DF9107
:10154000CF911F910F91FF90EF90DF90CF90089572
:10155000FC01538D448D252F30E0842F90E0821BB9
:10156000930B541710F0CF96089501970895FC013E
:10157000918D828D981761F0828DDF01A80FB11DCA
:101580005D968C91928D9F5F9F73928F90E00895EE
:101590008FEF9FEF0895FC01918D828D981731F0A8
:1015A000828DE80FF11D858D90E008958FEF9FEFFC
:1015B0000895FC01918D228D892F90E0805C9F4FD2
:1015C000821B91098F73992708958AE193E00E9405
:1015D000D90A21E0892B09F420E0822F0895FC012B
:1015E000848DDF01A80FB11DA35ABF4F2C91848DAC
:1015F00090E001968F739927848FA689B7892C93E1
:10160000A089B1898C9180648C93938D848D98137B
:1016100006C00288F389E02D80818F7D8083089544
:10162000EF92FF920F931F93CF93DF93EC0181E032
:10163000888F9B8D8C8D981305C0E889F9898081EE
:1016400085FD24C0F62E0B8D10E00F5F1F4F0F732A
:101650001127E02E8C8DE8120CC00FB607FCFACFD4
:10166000E889F989808185FFF5CFCE010E94EF0AD4
:10167000F1CF8B8DFE01E80FF11DE35AFF4FF08291
:101680000B8FEA89FB898081806207C0EE89FF8920
:101690006083E889F98980818064808381E090E0BB
:1016A000DF91CF911F910F91FF90EF900895CF930D
:1016B000DF93EC01888D8823C9F0EA89FB8980815A
:1016C00085FD05C0A889B9898C9186FD0FC00FB62C
:1016D00007FCF5CF808185FFF2CFA889B9898C916D
:1016E00085FFEDCFCE010E94EF0AE7CFDF91CF91CA
:1016F000089580E090E0892B29F00E94E50A81118D
:101700000C9400000895CF93DF931F92CDB7DEB7FE
:101710006983DC01ED91FC910280F381E02D41E0D1
:1017200050E0BE016F5F7F4F09950F90DF91CF9121
:10173000089583E08093E9008091F200882319F0F6
:101740008AE38093E80008950F931F93CF93DF936C
:101750001F92CDB7DEB782E0898342E450E06AECA5
:1017600070E080E80E94490A0E94591BDC01129631
:101770000D911C9113970115110569F0D801ED9198
:10178000FC910280F381E02DBE016F5F7F4FC801A5
:10179000099597FF07C089810F90DF91CF911F9125
:1017A0000F910895F80100851185E5CF8F929F92E2
:1017B000AF92BF92CF92DF92EF92FF920F931F935F
:1017C000CF93DF935C016B017A018091180188232C
:1017D00009F45BC080917B04882309F456C0809192
:1017E000660280FF05C08091E00082608093E00087
:1017F000E70110E00AEF83E0882E9AE3992E209704
:10180000D9F10E94481B81110AC0015009F43DC062
:1018100061E070E080E090E00E943A11F0CF282F64
:1018200030E0C217D3070CF48C2F4FB7F894809296
:10183000E9009091E80095FF1DC0282F30E0C21B01
:10184000D30BF601982F915020F081918093F100F5
:10185000FACFC20ED31E112319F09092E80009C0EE
:101860008091E80085FD06C09092E80011E0209785
:1018700009F010E04FBFC3CF1111C3CF5D9884E6CC
:10188000809393021E141F0444F081E090E0F50160
:101890009383828380E090E001C0C701DF91CF9104
:1018A0001F910F91FF90EF90DF90CF90BF90AF907E
:1018B0009F908F9008951F920F920FB60F92112450
:1018C0008F939F938091E1009091E100937F90939B
:1018D000E10083FF0FC01092E90091E09093EB00CC
:1018E0001092EC0092E39093ED0010927B0498E04C
:1018F0009093F00082FF20C093E09093E9009091D4
:10190000F200992319F09AE39093E80090919302E2
:10191000992339F0909193029150909393029923D7
:1019200089F190917A04992339F090917A04915039
:1019300090937A04992341F184FF10C08091E200D2
:101940008E7E81608093E2008091E1008F7E8093A3
:10195000E100809166028E7E806111C080FF16C01A
:101960008091E2008E7E80618093E2008091E100B0
:101970008E7E8093E100809166028E7E81608093EE
:10198000660204C05D9ACDCF289AD6CF9F918F91E1
:101990000F900FBE0F901F9018951F920F920FB6C9
:1019A0000F921124CF92DF92EF92FF920F931F9329
:1019B0002F933F934F935F936F937F938F939F9357
:1019C000AF93BF93EF93FF93CF93DF93CDB7DEB782
:1019D0006C97DEBFCDBF1092E9008091E80083FFD5
:1019E000EDC168E0CE0145960E94700A82EF8093B7
:1019F000E8008D8987FF05C09091E80090FFFCCF3B
:101A000003C09EEF9093E800982F907609F0C6C02F
:101A10009E892F89188D91110CC0803829F48091EE
:101A200067028093F10002C01092F1001092F10061
:101A300048C1422F50E0512B913051F4811141C1E6
:101A40004130510509F03DC1809167028D7F0BC087
:101A5000933061F4811135C14130510509F031C134
:101A6000809167028260809367022BC1953041F4B8
:101A70008091E80080FFFCCF20682093E30021C123
:101A8000963009F05FC0EB8CFC8C1092E90010924C
:101A9000920210929102123091F5109290021092DF
:101AA0008F020E94A40B99E0BE016F5F7F4FDB01A4
:101AB000E92F1D92EA95E9F799831A8391E09E83B5
:101AC00090EA98879AEF998720919102309192023B
:101AD000275F3F4F3C832B838D831092E900109248
:101AE000920210929102F0929002E0928F0249E0ED
:101AF00050E080E00E94490A0E94A40BE2C0F092EC
:101B00009002E0928F020E94591BDC011296ED9028
:101B1000FC901397E114F10409F4C0C0D701ED91D2
:101B2000FC910480F581E02DBE016B5E7F4FC70103
:101B30000995009719F00CF0C4C0C7C0F701E08404
:101B4000F184E8CF973009F4C0C0983021F481E0E7
:101B50008093F100B6C0993009F0B3C0837009F0EA
:101B6000B4C0E3E5F1E081E021E036E39081992320
:101B700061F08093E9002093EB0091919093EC0049
:101B80003093ED008F5F873089F78EE78093EA000E
:101B90001092EA008F8980937B0493C08B8D9C8D7B
:101BA0001092E9001092920210929102909390028A
:101BB00080938F02898D811156C08E899D89913ABB
:101BC00059F4813209F081C047E050E061E171E0F1
:101BD00080E00E94490A75C0913209F076C08332D4
:101BE00089F4888D90E0982F88272F89822BA0E098
:101BF000B0E080930D0190930E01A0930F01B0937C
:101C000010015FC0803269F48091E80082FFFCCF50
:101C100067E081E191E00E94700A8BEF8093E80019
:101C200006C0823209F04DC08F89809318018091DF
:101C30006502882319F0EEEFFAE002C0E0E0F8E078
:101C40008091110190911201A0911301B0911401A2
:101C5000803B9440A105B10509F07BC0809118013B
:101C600080FF93C076C00E94591BDC0112960D9133
:101C70001C9113970115110541F1D801ED91FC91CB
:101C80000190F081E02DBE016B5E7F4FC801099588
:101C9000811117C0F80100851185ECCF113009F4CE
:101CA0004EC0133091F48F89882309F445C08230E7
:101CB00081F440E860E18EE291E00E9400228823F6
:101CC00021F08EEF8093E80079C081E28093EB00F1
:101CD00075C0813029F440E86BE082E291E0EDCFFD
:101CE000833099F70E94591BDC011296ED90FC900D
:101CF00013978E010F5F1F4F6801E114F10479F013
:101D0000D701ED91FC910680F781E02DB801C70164
:101D10000995080F111DF701E084F184EECFD80179
:101D20001C92F60101900020E9F73197BF016C1970
:101D30007D0940E0C601C1CF6CE071E002C060E106
:101D400071E06115710509F2FB01449150E080E8F2
:101D500040CF0FB6F894A895809160008861809379
:101D60006000109260000FBEA895EE3F2AE0F207D7
:101D700039F08091FE0A9091FF0A91838083A1CF70
:101D80001092FF0A1092FE0A9CCFEE3F8AE0F807FD
:101D900031F0808191819093FF0A8093FE0A87E75A
:101DA00097E7918380839BE088E10FB6F894A8952C
:101DB000809360000FBE9093600083CF6C960FB647
:101DC000F894DEBF0FBECDBFDF91CF91FF91EF91B1
:101DD000BF91AF919F918F917F916F915F914F9143
:101DE0003F912F911F910F91FF90EF90DF90CF9037
:101DF0000F900FBE0F901F9018956115710579F027
:101E0000FB0101900020E9F73197AF01461B570B0A
:101E1000DC01ED91FC910280F381E02D099480E0DA
:101E200090E008951F920F920FB60F9211242F93F6
:101E30003F934F935F936F937F938F939F93AF9352
:101E4000BF93EF93FF938AE193E00E94EF0AFF9123
:101E5000EF91BF91AF919F918F917F916F915F9122
:101E60004F913F912F910F900FBE0F901F9018959B
:101E70001F920F920FB60F9211242F938F939F935F
:101E8000EF93FF93E0912A03F0912B038081E0917F
:101E90003003F091310382FD12C0908180913303B1
:101EA0008F5F8F7320913403821751F0E0913303D9
:101EB000F0E0E65EFC4F958F8093330301C0808194
:101EC000FF91EF919F918F912F910F900FBE0F90E7
:101ED0001F901895FC018485958597FD0BC09FB7D1
:101EE000F89482E08093E9008091F2009FBF90E037
:101EF000019608959FB7F89482E08093E90080915D
:101F0000F2009FBF90E0089590E0FC013197EF3020
:101F1000F105B0F5EA5AFF4F0C941125809180002D
:101F20008F7703C0809180008F7D8093800008951B
:101F300080918000877FF9CF84B58F7702C084B508
:101F40008F7D84BD0895809190008F7707C0809128
:101F500090008F7D03C080919000877F80939000D8
:101F600008958091C0008F7703C08091C0008F7D5D
:101F70008093C00008958091C200877F8093C20043
:101F8000089508952E98269A2D98259A2A98229A8F
:101F90002998219A80EA8093800081E180938100D2
:101FA00080E991E0909387008093860010928900E9
:101FB0001092880010928B0010928A0008954FB101
:101FC00041708CB186FB882780F984272091A0027C
:101FD00050919F026091980270919902982F9227D8
:101FE000292F30E0942F9527291B3109260F371F01
:101FF000309399022093980220919F029091A00221
:10200000821729F0491719F091E090939E0280936E
:102010009F024093A00208950E94481B90E00895FB
:102020000F931F93CF93DF931F92CDB7DEB78C0131
:10203000FC018485958597FF0EC0CE0101960E9414
:102040001E1B019719F4298130E002C02FEF3FEFEA
:10205000F80135872487F801848595850F90DF91F5
:10206000CF911F910F910895CF93DF931F92CDB71A
:10207000DEB7FC018485958597FD05C02FEF3FEF06
:10208000358724870BC0CE0101960E941E1B019745
:1020900019F4898190E002C08FEF9FEF0F90DF91DC
:1020A000CF910895CF93DF93282F30E0F901E955C0
:1020B000FE4F8491F901E857FE4FD491F901E75999
:1020C000FE4FC491CC2391F081110E94840FEC2F1C
:1020D000F0E0EE0FFF1FE55AFE4FA591B491EC9191
:1020E000ED2381E090E021F480E002C080E090E008
:1020F000DF91CF9108951F93CF93DF93282F30E086
:10210000F901E955FE4F8491F901E857FE4FD4914A
:10211000F901E759FE4FC491CC23C9F0162F811164
:102120000E94840FEC2FF0E0EE0FFF1FE35BFE4FE9
:10213000A591B4918FB7F894111105C09C91ED2F22
:10214000E095E92302C0EC91ED2BEC938FBFDF917A
:10215000CF911F910895CF93DF9390E0FC01E85752
:10216000FE4F2491FC01E759FE4F8491882361F1D1
:1021700090E0880F991FFC01E15CFE4FC591D4915E
:10218000FC01E35BFE4FA591B491611109C09FB7BB
:10219000F8948881209582238883EC912E230BC0AC
:1021A000623061F49FB7F8943881822F8095832341
:1021B0008883EC912E2B2C939FBF06C08FB7F89489
:1021C000E8812E2B28838FBFDF91CF910895CF9385
:1021D000DF93EC01888581110FC081E088878A85B3
:1021E000882311F062E001C060E089850E94AB1095
:1021F0008FE090E00197F1F789850E9452102B85BE
:1022000030E041E08217930709F440E0842FDF912A
:10221000CF9108958230910538F0880F991F880F6B
:10222000991F05970197F1F708953FB7F8948091AA
:10223000AA029091AB02A091AC02B091AD0226B57A
:10224000A89B05C02F3F19F00196A11DB11D3FBFEE
:10225000BA2FA92F982F8827820F911DA11DB11D7C
:10226000BC01CD0142E0660F771F881F991F4A9578
:10227000D1F708958F929F92AF92BF92CF92DF9243
:10228000EF92FF926B017C010E9415114B015C01E2
:10229000C114D104E104F104F1F00E941511DC0134
:1022A000CB0188199909AA09BB09883E9340A10569
:1022B000B10570F321E0C21AD108E108F10888EEF7
:1022C000880E83E0981EA11CB11CC114D104E10446
:1022D000F10419F7DDCFFF90EF90DF90CF90BF9022
:1022E000AF909F908F9008957F928F929F92AF9220
:1022F000BF92CF92DF92EF92FF920F931F93CF93F3
:10230000DF93FC0122853385232B09F479C07B01FF
:10231000EC01D12C8C85D816F0F40D2D10E08E85B3
:102320009F85F801EE0FFF1FEE0DFF1D9183808347
:10233000EA85FB85E00FF11F61E080810E947B1040
:102340008A859B85FC01E00FF11F61E080810E947E
:10235000AB10D394DFCF83E290E00197F1F710E068
:102360008C851817A8F4C12ED12CEA85FB85EC0DBD
:10237000FD1D60E080810E94AB108A859B85FC0179
:10238000EC0DFD1D60E080810E947B101F5FE8CF97
:102390000E9415114B015C010E941511AB01BC019B
:1023A000481959096A097B098E859F85A0E0B0E02C
:1023B000481759076A077B0718F50E9415116B012A
:1023C000C818D908712C8C85781630F7072D10E0C5
:1023D000EA85FB85E00FF11F80810E945210892B56
:1023E00051F4000F111FF701E00FF11F808191815F
:1023F000C816D90610F07394E6CFD182C082FBCF05
:10240000DF91CF911F910F91FF90EF90DF90CF90D0
:10241000BF90AF909F908F907F9008952FB7F894C2
:102420006091A6027091A7028091A8029091A902E2
:102430002FBF08951F920F920FB60F9211242F9362
:102440003F938F939F93AF93BF938091A6029091F8
:10245000A702A091A802B091A9023091A50223E0A1
:10246000230F2D3720F40196A11DB11D05C026E8CC
:10247000230F0296A11DB11D2093A5028093A602F1
:102480009093A702A093A802B093A9028091AA02F8
:102490009091AB02A091AC02B091AD020196A11D4A
:1024A000B11D8093AA029093AB02A093AC02B093AB
:1024B000AD02BF91AF919F918F913F912F910F905E
:1024C0000FBE0F901F9018951F920F920FB60F928C
:1024D00011242F933F934F935F936F937F938F9329
:1024E0009F93AF93BF93EF93FF93E0912201F091FD
:1024F00023010995FF91EF91BF91AF919F918F912A
:102500007F916F915F914F913F912F910F900FBEEF
:102510000F901F9018951F920F920FB60F921124D3
:102520002F933F934F935F936F937F938F939F93DB
:10253000AF93BF93EF93FF93E0912001F0912101BE
:102540000995FF91EF91BF91AF919F918F917F91ED
:102550006F915F914F913F912F910F900FBE0F9010
:102560001F9018951F920F920FB60F9211242F9360
:102570003F934F935F936F937F938F939F93AF930B
:10258000BF93EF93FF93E0911E01F0911F01099516
:10259000FF91EF91BF91AF919F918F917F916F913B
:1025A0005F914F913F912F910F900FBE0F901F9011
:1025B00018951F920F920FB60F9211242F933F93ED
:1025C0004F935F936F937F938F939F93AF93BF933B
:1025D000EF93FF93E0911C01F0911D010995FF918C
:1025E000EF91BF91AF919F918F917F916F915F918B
:1025F0004F913F912F910F900FBE0F901F90189504
:102600001F920F920FB60F9211242F933F934F9367
:102610005F936F937F938F939F93AF93BF93EF934A
:10262000FF93E0911A01F0911B010995FF91EF9141
:10263000BF91AF919F918F917F916F915F914F91DA
:102640003F912F910F900FBE0F901F9018950F93F1
:102650001F93CF93DF938C01EB018091A402811132
:1026600005C081E08093A4020E94C20F17FF05C03D
:1026700011950195110981E001C080E0013991E0D7
:10268000190714F000E911E010938B0000938A0001
:10269000882311F02A9A01C02A98229A8091A402D4
:1026A000811105C081E08093A4020E94C20FD7FF70
:1026B00005C0D195C195D10981E001C080E0C13943
:1026C00091E0D90714F0C0E9D1E0D0938900C0931C
:1026D0008800882311F0299A01C02998219ADF9156
:1026E000CF911F910F91089546983E9AE0E9F0E04E
:1026F00082E08083109291001092710010821092FB
:1027000099001092980010929700109296001092E3
:1027100095001092940086988E980895FC0110926E
:1027200071009B014617570708F49A0146983E9896
:1027300090E89093900010929100909392003E9AAE
:10274000EF2B11F08E9A01C08E98869A50939700C5
:102750004093960041505109509395004093940046
:10276000309399002093980082E88093900089E14B
:1027700080939100089524982C9A6A98729A6E9882
:10278000769A8098889A81E08093680090E190938F
:102790006B008BBB8FED9FE0909323018093220110
:1027A000EAE6F0E080818F7C80618083EE9A8CB1D4
:1027B00082FB882780F98093A30293B12091A30222
:1027C00094FB882780F982278093A20210929B02B3
:1027D00010929A021092A1028FB181708093A00290
:1027E0009CB12091A00296FB882780F982278093D4
:1027F0009F02109299021092980210929E020895E0
:102800001F920F920FB60F9211242F933F934F9365
:102810005F936F937F938F939F938CB190E0959587
:10282000879595958795482F417023B130E054E006
:10283000359527955A95E1F7822793278170209146
:10284000A3025091A20260919A0270919B02982F6C
:102850009227292F30E0942F9527291B3109260F25
:10286000371F30939B0220939A022091A2029091ED
:10287000A302821729F0491719F091E09093A10261
:102880008093A2024093A3029F918F917F916F91B9
:102890005F914F913F912F910F900FBE0F901F901E
:1028A000189580919D02E0919602F09197028823FD
:1028B00011F0849101C080819FEB980F9A3110F440
:1028C000805E0895803269F42091960230919702DB
:1028D000A9014F5F5F4F5093970240939602232BBD
:1028E00001F708951F93CF93DF930E945114C0E026
:1028F000D0E01AE090ED980F9A30B8F41C9F900148
:102900001D9F300D1124E901C80FD11D87FDDA95F7
:10291000E09780919602909197020196909397028A
:10292000809396020E945114E5CFCE01DF91CF91A2
:102930001F9108952F923F924F925F926F927F92D4
:102940008F929F92AF92BF92CF92DF92EF92FF92BF
:102950000F931F93CF93DF93CDB7DEB727970FB6B3
:10296000F894DEBF0FBECDBF9F838E831B014D83C6
:1029700080919C0281111BC081E080939C02109287
:1029800072001092C00094E09093C10099E090937F
:10299000C2008093C30083E08093BF0088EE8093E1
:1029A000D1001092BF001092D200579A78941092E2
:1029B00019012E813F8137FF05C03F773F832E836A
:1029C0000AE001C001E088E2089F802D112490E018
:1029D0004E815F814817590708F4C2C0013039F4AD
:1029E0004131574220F0E0E1F7E2FF83EE83802E91
:1029F000912CA12CB12C8E819F81969587959C015D
:102A000040E050E029833A834B835C834E815F81B1
:102A10002A01612C712CA501940160E072E18AE722
:102A200090E00E94CD2429813A814B815C81620F24
:102A3000731F841F951FA30192010E948B236901BC
:102A40007A01EE24FF2410E01F5FC11434E0D306A6
:102A5000E104F10408F120E032E14AE750E0012E00
:102A600004C055954795379527950A94D2F7C50127
:102A7000B4010E94CD2429813A814B815C81620F8F
:102A8000731F841F951FA30192010E948B2369016C
:102A90007A01EE24FF24D8CF0A3049F48E819F8139
:102AA00005966AE070E00E94E9247F836E834E8180
:102AB0005F81483E83E0580759F09101DA010E9496
:102AC000162428EE33E040E050E00E948B231901E9
:102AD000109272008091C100807F182B1093C1006A
:102AE000BB27AF2D9E2D8D2D8093BF00C092D100AE
:102AF0002D81203108F02FE080E190E0821B9109C8
:102B000004C0F694E794D794C7948A95D2F78D2D94
:102B100099278093BF00C092D200309295022092F4
:102B2000940289B38FEF89BB84E08093720027966B
:102B30000FB6F894DEBF0FBECDBFDF91CF911F91CE
:102B40000F91FF90EF90DF90CF90BF90AF909F904C
:102B50008F907F906F905F904F903F902F9008954F
:102B60009F838E8344CF40916E0420916C043091FA
:102B70006D0490E0941749F02D5F3F4FF9013397B2
:102B80005081581721F09F5FF5CF8FEF0895892F5F
:102B900008952091190390917904213208F04AC0D8
:102BA0008091F6028111FCCF32E03093F60231E0E1
:102BB0003093F5023FEF3093F4021092F30220932A
:102BC000F202A9EFB2E042ED52E0FA013E2F341BCF
:102BD000321718F43D913193F9CF1092D102209120
:102BE000D102990F922B9093D1029091D002913003
:102BF00061F41092D0029091D1029093BB00909119
:102C0000BC0093FDF8CF95EC01C095EE9093BC000D
:102C10009091F6029230E1F39091F4029F3F79F0A7
:102C20008091F402803241F08091F402803331F0DF
:102C300084E005C081E003C082E001C083E010921F
:102C4000F802109219031092F702089591E0909300
:102C5000F702809379041092F802109219030895F4
:102C60009091F6029111FCCF613208F060E291E0A0
:102C70009093F6029093F5022FEF2093F4021092B6
:102C8000F302260F2093F2029093D1029091D10289
:102C9000880F892B8093D1028091D002813061F41A
:102CA0001092D0028091D1028093BB008091BC0031
:102CB00083FDF8CF85EC01C085EE8093BC00809148
:102CC000F6028130E1F38091F302861710F46091EF
:102CD000F302A2EDB2E020EB32E0F9018E2F821B6D
:102CE000861718F48D918193F9CF1092AF026093FB
:102CF000AE02862F0895CF93C82F0E9426166FE04C
:102D000087E094E00E949D010E94C91581110FC0C7
:102D100061E08C2F0E9430169091AE028091AF023C
:102D2000981729F087E094E0CF910C9451018FEF30
:102D30009FEFCF910895BF92CF92DF92EF92FF92D3
:102D40000F931F93CF93DF9380911C040E9426164C
:102D500068EA87E094E00E949D010E94C91566E040
:102D600080911C040E9430160E940E127B018091FB
:102D7000AE0290E02091AF02821B91090697ACF45D
:102D800080911D0490911E04892B89F30E940E12DC
:102D90006E197F0980911D0490911E048617970774
:102DA00030F781E080931F0433C087E094E00E94F5
:102DB0005101C82E87E094E00E945101B82E87E0AF
:102DC00094E00E945101E82E87E094E00E945101B6
:102DD000D82E87E094E00E945101F82E87E094E01D
:102DE0000E9451011B2D00E00C2910931404009344
:102DF0001304DD2D20E0C22FCE29D0931604C093FA
:102E00001504982F88278F2990931804809317040E
:102E1000DF91CF911F910F91FF90EF90DF90CF90B6
:102E2000BF9008950F931F93CF93DF93082F162F12
:102E3000C3E1D4E089850E942616602F87E094E0E4
:102E40000E949D01612F87E094E00E949D010E94F5
:102E5000C9158E83DF91CF911F910F910895CF9364
:102E6000DF93BC0187EB93E00E94FD0EEC016DE067
:102E700072E087EB93E00E94FD0E8C0F9D1FDF91A7
:102E8000CF9108958BE60E947B168F3F2FEF92071C
:102E900081F48AE60E947B168F3F2FEF920761F440
:102EA00089E60E947B16833D910541F521E030E0E3
:102EB0002DC021E030E002C020E030E0873D9105E8
:102EC000D1F081E090E090931B0480931A04019765
:102ED000029738F42130310511F08AE608C08BE6FC
:102EE00006C02130310511F088E601C089E68093E3
:102EF0001C0481E0089582E090E0E5CF88E60E941E
:102F00007B16833D910529F420E030E080E090E0DD
:102F1000DACF80E00895EF92FF920F931F93CF9343
:102F2000DF9380913C040E94261680913904909191
:102F30003A04039731F4609141047091420460684F
:102F400004C060913F047091400487E094E00E94C7
:102F50009D010E94C9158093380466E080913C046D
:102F60000E9430160E940E12EB018091AE0290E09A
:102F70002091AF02821B91090697ACF480914B041B
:102F800090914C04892B89F30E940E126C1B7D0BCF
:102F900080914B0490914C048617970730F781E09D
:102FA00080934D0474C08091390490913A04039742
:102FB000F9F487E094E00E945101182F87E094E033
:102FC0000E945101E82E87E094E00E945101D82F21
:102FD00087E094E00E945101F82E87E094E00E947F
:102FE0005101C82F87E094E00E945101082F39C099
:102FF00087E094E00E945101E82E87E094E00E946F
:103000005101182F8091390490913A04892BA9F429
:1030100087E094E00E945101F82E87E094E00E943E
:103020005101D82F87E094E00E945101082F87E0DA
:1030300094E00E945101C82F14C087E094E00E94E0
:103040005101082F87E094E00E945101C82F87E0CA
:1030500094E00E945101F82E87E094E00E94510113
:10306000D82F212F30E03E293093270420932604C7
:103070002D2F30E03F2930932904209328042C2F52
:1030800030E0C901902B90932B0480932A04DF91A8
:10309000CF911F910F91FF90EF900895BF92CF9223
:1030A000DF92EF92FF920F931F93CF93DF93809164
:1030B0003B040E94261668EA87E094E00E949D0186
:1030C0000E94C9158093380466E080913B040E94F9
:1030D00030160E940E127B018091AE0290E020918A
:1030E000AF02821B91090697ACF480914B0490913A
:1030F0004C04892B89F30E940E126E197F0980916E
:103100004B0490914C048617970730F781E0809329
:103110004D0433C087E094E00E945101C82E87E03F
:1031200094E00E945101B82E87E094E00E94510182
:10313000E82E87E094E00E945101D82E87E094E0C9
:103140000E945101F82E87E094E00E9451011B2D4E
:1031500000E00C291093210400932004DD2D20E0D1
:10316000C22FCE29D0932304C0932204982F8827FE
:103170008F299093250480932404DF91CF911F9190
:103180000F91FF90EF90DF90CF90BF9008950F9335
:103190001F93CF93DF93082F162FC0E2D4E08C8DBE
:1031A0000E942616602F87E094E00E949D01612F07
:1031B00087E094E00E949D010E94C915888FDF91ED
:1031C000CF911F910F9108950F931F93CF93DF938A
:1031D000082F162FC0E2D4E08B8D0E942616602F98
:1031E00087E094E00E949D01612F87E094E00E94B7
:1031F0009D010E94C915888FDF91CF911F910F917A
:1032000008952091390430913A042330310511F0AA
:10321000803210F40C94C7180C94E4181F93CF93C9
:10322000DF931F92CDB7DEB7182F69830E94261651
:10323000698187E094E00E949D010E94C915811177
:1032400012C061E0812F0E9430169091AE028091F1
:10325000AF02981741F087E094E00F90DF91CF9193
:103260001F910C9451018FEF9FEF0F90DF91CF9141
:103270001F910895809167048F3F61F061E00E9483
:10328000AB1060E0809167040E947B108BE193E0BB
:103290000197F1F708956FE070E08DE10E940E193B
:1032A0008934910561F06FE070E08EE10E940E19A3
:1032B0008934910509F0A2C020E030E002C021E08D
:1032C00030E083E090E090933A04809339048230B8
:1032D000910539F589E180933B048EE180933C04AC
:1032E00083E090E09093400480933F0484E090E07A
:1032F000909342048093410487E090E090934404CB
:103300008093430488E090E09093460480934504C2
:1033100085E090E0909348048093470486E090E035
:1033200030C08330910599F1019709F45FC02130D5
:10333000310509F461C088E180933B048EE18093FC
:103340003C0483E090E09093400480933F0484E049
:1033500090E0909342048093410485E090E0909344
:1033600044048093430486E090E090934604809365
:10337000450487E090E0909348048093470488E0F8
:1033800090E090934A048093490481E008952130AD
:10339000310511F08EE101C08DE180933C048093F2
:1033A0003B0488E090E0909342048093410489E0DC
:1033B00090E09093400480933F048AE090E09093E3
:1033C0004604809345048BE090E0909344048093FE
:1033D00043048CE090E090934A04809349048DE08C
:1033E00090E09093480480934704CFCF213031057B
:1033F00009F470CF88E16FCF89E19ECF60E270E081
:1034000089E10E940E19019661F06FE070E08EE193
:103410000E940E1921E030E0CC97D9F080E090E0D6
:1034200052CF60E270E088E10E940E19019679F0B7
:103430006FE070E08EE10E940E1931E020E0CC9741
:1034400009F030E0832F922F20E030E03CCF80E085
:10345000089582E090E037CFFF920F931F93CF93B0
:10346000DF93CDB7DEB7A0970FB6F894DEBF0FBEDF
:10347000CDBF8C01F62E8FEF860F823088F48091BD
:1034800067048F3F79F061E00E94AB1061E08091AA
:1034900067040E947B108BE193E00197F1F702C073
:1034A0000E943A19E0915A04F0915B040190F08176
:1034B000E02DB8018AE594E009950E943A1962E08E
:1034C000F61231C0E0915A04F0915B040190F08152
:1034D000E02DBE016F5F7F4F8AE594E0099540E0E3
:1034E000809166044817F8F4242F30E0220F331F30
:1034F000F801E20FF31FA1E0B0E0AC0FBD1FA20F77
:10350000B31F80916804909169042D913C91BC0196
:10351000621B730B9B0180819181280F391F3183BE
:1035200020834F5FDDCFA0960FB6F894DEBF0FBEAD
:10353000CDBFDF91CF911F910F91FF9008958F9292
:103540009F92AF92BF92CF92DF92EF92FF920F9332
:103550001F93CF93DF93CDB7DEB7A1970FB6F89443
:10356000DEBF0FBECDBF6C01990FEE08FF08F7FE5E
:1035700033C0E0911A03F0911B030190F081E02D1C
:103580006DE28AE193E009958C0122273327A90196
:103590002C193D094E095F0919A2CE0181967C01C3
:1035A0009AE0892E912CA12CB12CCA01B901A50158
:1035B00094010E94F423605DF70162937F0121155D
:1035C00031054105510589F7BF018AE193E00E9469
:1035D000FD0E800F911F1FC0A701960119A28E0139
:1035E0000F5D1F4F8AE0C82ED12CE12CF12CCA01AF
:1035F000B901A70196010E94F423605DF80162936E
:103600008F01211531054105510589F7BF018AE177
:1036100093E00E94FD0EA1960FB6F894DEBF0FBE98
:10362000CDBFDF91CF911F910F91FF90EF90DF9071
:10363000CF90BF90AF909F908F900895FC018091A4
:103640007B04811103C08FEF9FEF08959FB7F8941B
:1036500082E08093E9002091F20030E01216130618
:1036600014F421E030E02115310559F0289884E662
:1036700080937A048091F10080838091F200882306
:1036800019F09FBFC90108958BE68093E800F9CF38
:103690002FB7F89483E08093E9009091E800892F98
:1036A000807295FF04C09091F20080E4891B2FBFC7
:1036B00008958091800481110DC082E080937C0484
:1036C00084E080937D0410927F0410927E0481E058
:1036D000809380048CE794E008958BEA91E09093C6
:1036E0005B0480935A048091640490916504009770
:1036F00011F00E94962680915E0490915F040097DD
:1037000011F00E94962680916204909163040097C4
:1037100011F00E94962680915C0490915D040097C0
:1037200011F00E94962680916004909161040097A8
:1037300011F00C9496260895CF93DF93CDB7DEB7A2
:10374000CB56D1090FB6F894DEBF0FBECDBF78942B
:1037500084B5826084BD84B5816084BD85B5826096
:1037600085BD85B5816085BD80916E008160809347
:103770006E001092810080918100826080938100B0
:1037800080918100816080938100809180008160C0
:10379000809380008091910082608093910080915D
:1037A000910081608093910080919000816080936E
:1037B00090008091C10084608093C1008091C1001D
:1037C00082608093C1008091C10081608093C100BC
:1037D0008091C30081608093C3008091C0008260AB
:1037E0008093C0008091C20081608093C20080916C
:1037F0007A00846080937A0080917A00826080935E
:103800007A0080917A00816080937A0080917A00BA
:10381000806880937A0010927B0410926702109265
:1038200066028091D70081608093D70080EA809300
:10383000D80089B5806189BD89B5826089BD09B428
:1038400000FEFDCF61E070E080E090E00E943A1160
:103850008091D8008F7C80618093D8008091E000B7
:10386000807F8093E0008091E1008E7E8093E10074
:103870008DE08093E200559A209AEEEFFFE7859164
:1038800094918B3F9C4D19F481E080936502E09107
:103890002A03F0912B0382E08083E0912603F091CC
:1038A00027031082E0912803F09129038FEC808395
:1038B00010923203E0912E03F0912F0386E0808373
:1038C000E0912C03F0912D03808180618083E09151
:1038D0002C03F0912D03808188608083E0912C037C
:1038E000F0912D03808180688083E0912C03F0911A
:1038F0002D0380818F7D80838AE090E0A0E0B0E09E
:1039000080931E0390931F03A0932003B093210381
:103910008AE193E00E94D90A892B21F083EB91E0A0
:103920000E942F178AE193E00E94D90A18161906FF
:1039300024F48AE193E00E94B70A1092AF02109239
:10394000AE021092F802109219031092F60281E072
:103950008093F5021092D00261E082E00E947B1019
:1039600061E083E00E947B108091B9008E7F80939C
:10397000B9008091B9008D7F8093B90088E480936D
:10398000B80085E48093BC0064EF71E080E090E0D3
:103990000E943A118BE080936F0469E070E080919F
:1039A0006C0490916D040E942E27FC01009769F031
:1039B00090936D0480936C0483E080936E0484E1A3
:1039C000808386E1838384E0868381E00E943B07D5
:1039D00082E1898385E18A838CE08B8310925D0488
:1039E00010925C0410925F0410925E0410926104C5
:1039F00010926004109263041092620410926B049F
:103A000010926A0483E0809366048091640490912C
:103A10006504892B11F080E00BC083E090E00E94E8
:103A200001269093650480936404892BA1F719C043
:103A300090916604891790F4282F30E0E091640497
:103A4000F0916504E20FF31FA1E0B0E0AC0FBD1FE1
:103A5000A20FB31F9C9190838F5FEACF8BE080937E
:103A6000670480ED97E0909369048093680431EED9
:103A7000A2963FAFA297412C512C3201812C912C60
:103A80005401C12CD12C7601A2964FADA2974C3394
:103A900028F46CE97FEF8AE690E004C064E670E009
:103AA00086E99FEF0E94271361E088E692E00E947A
:103AB0002C1A8091680290916902C80ED91EE11CEF
:103AC000F11C80916A0290916B02880E991EA11CD4
:103AD000B11C80916C0290916D02480E591E611CC0
:103AE000711C80915E0490915F04892B39F0809164
:103AF0005C0490915D04892BD1F41CC00091660494
:103B000010E0C801880F991F0E94012690935F045E
:103B100080935E04009709F4C5C0FC0180E090E04A
:103B20008017910724F7119211920196F9CF00E0C6
:103B300010E01DC00091660410E0C801880F991FB5
:103B40000E94012690935D0480935C04009709F421
:103B5000A9C02091680430916904FC0180E090E0E4
:103B60008017910724F7219331930196F9CF61E0F3
:103B7000CE018F5B9F4F0E942C1A80916604A82F64
:103B8000B0E0A696BFAFAEAFA697FE013196A49661
:103B9000FFAFEEAFA497E05CFF4F9E012F5D3F4F5C
:103BA0001901AC963FAF2EAFAC97AE014F5F5F4FA0
:103BB00060E070E0A6968EAD9FADA6976817790776
:103BC000BCF501151105A1F0AC96AEADBFADAC973B
:103BD0002D913C91808191812817390748F0DA01B5
:103BE0002D913C91808191818217930760F010C0E4
:103BF00080819181AC96AEADBFADAC978D939C9317
:103C00000115110561F780819181DA018D939C93F3
:103C10006F5F7F4F4E5F5F4F3296AC962EAD3FADDC
:103C2000AC972E5F3F4FAC963FAF2EAFAC97C2CF55
:103C30000F5F1F4F0A30110509F099CFA0915C0466
:103C4000B0915D0460915E0470915F0480E090E04B
:103C50002091660430E08217930724F5A496EEAD18
:103C6000FFADA49721913191A496FFAFEEAFA49739
:103C7000FB01408151814217530710F431832083A7
:103C8000F101219131911F014D915C911197241700
:103C9000350718F411963C932E93019612966E5F99
:103CA0007F4FD6CFA2962FADA2972F5FA2962FAFB0
:103CB000A297293509F0E8CE60E070E080E090E05E
:103CC0000E942713C701B60128E730E040E050E02A
:103CD0000E94F4233093690220936802C501B40165
:103CE00028E730E040E050E00E94F42330936B027C
:103CF00020936A02C301B20128E730E040E050E0BF
:103D00000E94F42330936D0220936C0280E00E94A5
:103D10003B0781E00E943B070E9442170E94421726
:103D200081110DC02898209A83ED91E00E942F17F1
:103D300068E873E180E090E00E943A11F5CF6FEF00
:103D400080E20E94121760E283E20E94121760E094
:103D500084E20E94121700E014E0C12CD12C7601FD
:103D600080911C040E94261667E287E094E00E947E
:103D70009D010E94C9158093190461E080911C0483
:103D80000E94301687E094E00E9451010E94C915FC
:103D90000E949B168091170490911804092E000C24
:103DA000AA0BBB0BC80ED91EEA1EFB1E015011093F
:103DB000B9F6C701B60120E034E040E050E00E94CF
:103DC0008B2330937102209370020E94151170931F
:103DD0006F0260936E0280E00E943B0781E00E94C8
:103DE0003B070E944B190E944B1981110DC0289866
:103DF000209A8FEE91E00E942F1768E873E180E02F
:103E000090E00E943A11F5CF8091390490913A04E4
:103E100083309105A9F460E081E20E94011967E511
:103E200080E20E94011964E684E20E94011960E2C6
:103E300085E20E94011960E086E20E9401191CC01F
:103E4000029731F468E083E20E94E41867E405C059
:103E500060E083E20E94E41867E280E20E94E418D6
:103E60006CE080E00E94C71860E281E00E94C71801
:103E700060E082E00E94C71800E014E060E070E0BB
:103E8000CB01A7966FAFA797A8967FAFA897A996E3
:103E90008FAFA997AA969FAFAA970E944E180E942B
:103EA0008B17C0902004D09021040D2C000CEE083C
:103EB000FF08A7966FADA797A8967FADA897A9967C
:103EC0008FADA997AA969FADAA976C0D7D1D8E1DEB
:103ED0009F1D01501109A9F620E034E040E050E0B8
:103EE0000E948B23309389022093880280E00E94F5
:103EF0003B075D98559AE0914E04F0914F04019074
:103F0000F081E02D8EE494E009958823A1F36AE026
:103F100070E080E090E00E943A11E0914E04F09150
:103F20004F040190F081E02D8EE494E00995882300
:103F300011F3E0914E04F0914F040190F081E02DD7
:103F40008EE494E009958111F4CF6AE070E080E09E
:103F500090E00E943A11E0914E04F0914F040190DC
:103F6000F081E02D8EE494E009958111E2CF0E946A
:103F70000E12611571058105910511F00E94312322
:103F800064EF71E080E090E00E943A1111E0C12CF2
:103F9000D12C80E8E82E8FE3F82E93E3892E982C1D
:103FA00093EBA92E9FE3B92E5D9A559A80E00E946B
:103FB0003B07289A209A0E94DC050E94FA040E947E
:103FC00031050E944E180E948B1780912004909119
:103FD00021042091880230918902821B930B9093D7
:103FE0008B0280938A020E94A6050E942E078AE116
:103FF00093E00E94D90A1816190644F48AE193E066
:104000000E94B70A90938E0280938D0280918D0258
:1040100090918E028133910519F410938C0204C0A3
:10402000C09711F410928C0280918C028823A1F128
:104030008092090190920A01A0920B01B0920C01AA
:1040400080918A0290918B028D3D9540ECF4809195
:104050008502863021F4809186028630A9F0809115
:104060007E0290917F02853F914074F4809182029C
:1040700090918302853F91403CF480918002909121
:104080008102853691052CF060E070E080E090E0E0
:1040900055C10E944207B1C1C0920901D0920A01E4
:1040A000E0920B01F0920C0180918502863009F0BC
:1040B00048C180918602863009F043C181E090E0DA
:1040C0000E949F1A81E00E943B0710927602109294
:1040D0007702109278021092790210927202109276
:1040E000730210927402109275020E943105809141
:1040F000720290917302A0917402B09175028D9733
:10410000A105B1059CF40E9431050E94A60564E654
:1041100070E08BE190E00E942713809182029091E1
:104120008302895791098B37914008F70E94A605B1
:104130008091820290918302883791054CF40E940D
:10414000A60564E670E08AE690E00E942713F0CFAF
:104150000E9431058091720290917302A0917402C5
:10416000B09175020B97A105B1051CF10E943105B4
:104170000E94A60580917E0290917F028759910945
:104180008D35914018F460E070E00EC0809182029D
:1041900090918302895791098B37914018F464E616
:1041A00070E002C069E170E08AE690E00E942713A7
:1041B000D1CF64E670E08AE690E00E9427130E9467
:1041C000DC050E940E1270937D0260937C02809148
:1041D0008702863080F480917A0290917B02883B3E
:1041E0009B4048F40E942E070E94DC050E94A60511
:1041F0000E944207ECCF0E94DC0580918702863046
:1042000039F40E94DC050E94A6050E944207F5CF02
:104210000E940E1270937D0260937C020E942E0712
:1042200080917A0290917B02883B9B4038F40E94F7
:104230002E070E94A6050E944207F2CF1092760236
:104240001092770210927802109279021092720204
:104250001092730210927402109275020E9431053E
:104260008091720290917302A0917402B0917502D4
:10427000843D9F4FAF4FBF4F9CF00E9431050E947D
:10428000A60569E170E08AE690E00E94271380911C
:104290007E0290917F02875991098D35914000F7F8
:1042A0000E94A60580917E0290917F028639910539
:1042B0004CF40E94A60564E670E08AE690E00E9455
:1042C0002713F0CF0E943105809172029091730202
:1042D000A0917402B0917502863F9F4FAF4FBF4FC0
:1042E0002CF50E9431050E94A605809182029091D2
:1042F0008302895791098B37914028F464E670E076
:1043000080E090E010C080917E0290917F028759FA
:10431000910964E670E08D35914018F48AE690E0EA
:1043200002C08BE190E00E942713CECF80E090E0A6
:104330000E949F1A64E670E08AE690E00E942713CC
:104340005CC020917E0230917F02255F31408091D8
:104350008002909181022338334048F49C012D5211
:1043600031402F38314018F40E94180846C020917F
:10437000820230918302255F31402338334030F48C
:104380009C012D5231402F38314070F385569109F0
:10439000873C910508F07DCE2898209A81E090E036
:1043A0000E949F1A0E940E1270937D0260937C02FD
:1043B00080917E0290917F02863991052CF080E0F9
:1043C00090E00E949F1A19C080918202909183020E
:1043D00088379105A4F70E942E070E94A6056CE974
:1043E0007FEF86E99FEF0E94271380917A029091D8
:1043F0007B02893B9B40E0F2E2CF0E94790BD4CD57
:10440000CF92DF92EF92FF920F931F93CF93DF93A0
:104410001F92CDB7DEB7182F062FE42E862F880FF8
:104420008E5F99830E941B0A83E00E941B0AF12E73
:10443000C12E9981D92E8C2D8F19801798F4F601F1
:10444000E7FE02C0849101C080810E941B0A182FE0
:1044500080E00E941B0A8123FFEFCF1ADF0A81113F
:10446000EACF01C081E00F90DF91CF911F910F91B2
:10447000FF90EF90DF90CF900895EAE1F3E0138290
:10448000128288EE93E0A0E0B0E084839583A68357
:10449000B78329E631E0318320832DEC30E0358786
:1044A00024872CEC30E03787268728EC30E0318BEE
:1044B000208B29EC30E0338B228B2AEC30E0358BDB
:1044C000248B2EEC30E0378B268B118E128E138EC0
:1044D000148EE7EBF3E01382128284839583A68324
:1044E000B7832BE731E0318320832FEF3FEF358710
:1044F0002487E7E0F4E01382128284839583A68305
:10450000B7838DE891E091838083ECE6F4E011823B
:10451000108212828FEF838315821482168285EABD
:1045200091E09287818782E492E09487838784EA8E
:1045300091E090878783EAE5F4E013821282158286
:10454000148217821682118610861386128681EBDA
:1045500091E091838083EEE4F4E01282158210866C
:104560008EE0818781E0828783878FE991E0918364
:10457000808386E0E9E5F1E0A2E3B4E001900D92EA
:104580008A95E1F786E0EFE5F1E0ACE2B4E0019076
:104590000D928A95E1F7E0E2F4E084E090E0928FFA
:1045A000818F14A613A615A6E3E1F4E083E090E062
:1045B0009087878313861286148608958F929F9220
:1045C000AF92BF92CF92DF92EF92FF92CF93DF93A1
:1045D000EC01688179818A819B8161157105810572
:1045E000910521F464E279ED8BE597E02DE133EF5D
:1045F00041E050E00E948B2349015A019B01AC012C
:10460000A7EAB1E40E94AA236B017C01ACEEB4EFEF
:10461000A50194010E94B823DC01CB018C0D9D1DE6
:10462000AE1DBF1DB7FF03C00197A109B048888325
:104630009983AA83BB83BC01CD019F77DF91CF9182
:10464000FF90EF90DF90CF90BF90AF909F908F90B2
:1046500008950E94DE22089584E291E00E94DE2205
:10466000089560932401709325018093260190930F
:104670002701089597F99F6780E870E060E008954A
:104680009FEF80EC089500240A941616170618066A
:104690000906089500240A94121613061406050646
:1046A0000895092E0394000C11F4882352F0BB0FD7
:1046B00040F4BF2B11F460FF04C06F5F7F4F8F4F3A
:1046C0009F4F089557FD9058440F551F59F05F3F75
:1046D00071F04795880F97FB991F61F09F3F79F024
:1046E00087950895121613061406551FF2CF4695A6
:1046F000F1DF08C0161617061806991FF1CF869528
:104700007105610508940895E894BB27662777270B
:10471000CB0197F90895052E97FB1EF400940E9493
:10472000A22357FD07D00E94F42307FC03D04EF4C8
:104730000C94A22350954095309521953F4F4F4FB3
:104740005F4F089590958095709561957F4F8F4F3D
:104750009F4F08950E941624A59F900DB49F900D21
:10476000A49F800D911D11240895B7FF0C94AA23D6
:104770000E94AA23821B930B08952F923F924F927F
:104780005F926F927F928F929F92AF92BF92CF92E1
:10479000DF92EF92FF920F931F93CF93DF93CDB7EA
:1047A000DEB7CA1BDB0B0FB6F894DEBF0FBECDBF62
:1047B00009942A88398848885F846E847D848C8433
:1047C0009B84AA84B984C884DF80EE80FD800C813C
:1047D0001B81AA81B981CE0FD11D0FB6F894DEBF1F
:1047E0000FBECDBFED010895A1E21A2EAA1BBB1B7F
:1047F000FD010DC0AA1FBB1FEE1FFF1FA217B307AD
:10480000E407F50720F0A21BB30BE40BF50B661FC2
:10481000771F881F991F1A9469F760957095809586
:1048200090959B01AC01BD01CF010895A29FB001FD
:10483000B39FC001A39F700D811D1124911DB29FD4
:10484000700D811D1124911D08950E9439240C942E
:1048500051230E944A2358F00E94432340F029F438
:104860005F3F29F00C943A2351110C9485230C944A
:1048700040230E94622368F39923B1F3552391F3F7
:10488000951B550BBB27AA2762177307840738F0BF
:104890009F5F5F4F220F331F441FAA1FA9F335D01C
:1048A0000E2E3AF0E0E832D091505040E695001CD0
:1048B000CAF72BD0FE2F29D0660F771F881FBB1F8A
:1048C000261737074807AB07B0E809F0BB0B802D68
:1048D000BF01FF2793585F4F3AF09E3F510578F094
:1048E0000C943A230C9485235F3FE4F3983ED4F371
:1048F000869577956795B795F7959F5FC9F7880F68
:10490000911D9695879597F90895E1E0660F771FB9
:10491000881FBB1F621773078407BA0720F0621B4A
:10492000730B840BBA0BEE1F88F7E09508950E9475
:104930009E246894B1110C94852308950E946A23E3
:1049400088F09F5798F0B92F9927B751B0F0E1F050
:10495000660F771F881F991F1AF0BA95C9F714C000
:10496000B13091F00E948423B1E008950C94842327
:10497000672F782F8827B85F39F0B93FCCF3869539
:1049800077956795B395D9F73EF490958095709596
:1049900061957F4F8F4F9F4F0895DB018F939F93BA
:1049A0000E94AA23BF91AF91A29F800D911DA39F4A
:1049B000900DB29F900D11240895991B79E004C0C9
:1049C000991F961708F0961B881F7A95C9F780954E
:1049D0000895AA1BBB1B51E107C0AA1FBB1FA61746
:1049E000B70710F0A61BB70B881F991F5A95A9F798
:1049F00080959095BC01CD01089597FB072E16F484
:104A0000009407D077FD09D00E94E92407FC05D067
:104A10003EF4909581959F4F0895709561957F4FD5
:104A20000895EE0FFF1F0590F491E02D09940E9468
:104A30001624B7FF0895821B930B089597FB57FF29
:104A40000C942E259F938F930E942E256E1B7F0B17
:104A5000AF91BF918A0B9B0B0895E894DF93CF939E
:104A6000FC01DB010E9416247F936F93E9019A01F8
:104A7000AC01BF93AF933F932F93DF010E941624A5
:104A800026F46C1B7D0B820B930B9E01EB01FC014A
:104A90000E94F825AF91BF912F913F910E94F82578
:104AA000BE01CF01F9012F913F91CF91DF91089580
:104AB000689401C0E894F92FF12B12F00C948C2526
:104AC000A0E0B0E0E6E6F5E20C94C323092E0594DD
:104AD00022F40E94E825112392F4F0E80F26FFEF5C
:104AE000E094F09400951095B094C094D094A19463
:104AF000BF0ACF0ADF0AEF0AFF0A0F0B1F0B0E9443
:104B0000972507FC0E94E825CDB7DEB7ECE00C94B2
:104B1000DF23689401C0E8948F929F92CF93DF9334
:104B20000E949725DF91CF919F908F9008958824C0
:104B30009924F401E401B0E49F93AA279A158B0409
:104B40009C04ED05FE05CF05D007A10798F4AD2F15
:104B5000DC2FCF2FFE2FE92D982C892E982F872F11
:104B6000762F652F542F432F322F2227B85031F73D
:104B7000BF9127C01B2EBF91BB27220F331F441F9D
:104B8000551F661F771F881F991F881C991CEE1FD1
:104B9000FF1FCC1FDD1FAA1FBB1F8A149B04EC053F
:104BA000FD05CE05DF05A007B10748F08A189B0870
:104BB000EC09FD09CE09DF09A00BB10B21601A94A5
:104BC000E1F62EF49401AF01BE01CD01000C089571
:104BD000609570958095909530954095509521956C
:104BE0003F4F4F4F5F4F6F4F7F4F8F4F9F4F0895F6
:104BF0000E941624460F571FC81FD91F08F431966C
:104C00000895CF93DF938230910510F482E090E015
:104C1000E0918A04F0918B0420E030E0C0E0D0E025
:104C2000309711F14081518148175907C0F048175A
:104C3000590761F482819381209719F09B838A83BD
:104C40002BC090938B0480938A0426C021153105D4
:104C500019F04217530718F49A01BE01DF01EF0162
:104C60000280F381E02DDCCF2115310509F1281BED
:104C7000390B2430310590F412968D919C91139745
:104C80006115710521F0FB019383828304C0909329
:104C90008B0480938A04FD01329644C0FD01E20F2B
:104CA000F31F81939193225031092D933C933AC085
:104CB0002091880430918904232B41F420912A010A
:104CC00030912B013093890420938804209128018E
:104CD000309129012115310541F42DB73EB740919E
:104CE0002C0150912D01241B350BE0918804F0918B
:104CF0008904E217F307A0F42E1B3F0B281739078E
:104D000078F0AC014E5F5F4F2417350748F04E0F27
:104D10005F1F50938904409388048193919302C04C
:104D2000E0E0F0E0CF01DF91CF9108950F931F9362
:104D3000CF93DF93009709F48CC0FC013297138264
:104D4000128200918A0410918B040115110581F4DF
:104D500020813181820F931F209188043091890432
:104D60002817390779F5F0938904E093880471C016
:104D7000D80140E050E0AE17BF0750F412962D91D5
:104D80003C911397AD012115310509F1D901F3CFFC
:104D90009D01DA013383228360817181860F971F21
:104DA0008217930769F4EC0128813981260F371F98
:104DB0002E5F3F4F318320838A819B81938382833F
:104DC000452B29F4F0938B04E0938A0442C0139698
:104DD000FC93EE931297ED01499159919E01240F96
:104DE000351FE217F30771F480819181840F951FBD
:104DF000029611969C938E938281938113969C9335
:104E00008E931297E0E0F0E0D80112968D919C917C
:104E10001397009719F0F8018C01F6CF8D919C91B2
:104E200098012E5F3F4F820F931F2091880430918D
:104E300089042817390769F4309729F410928B04F4
:104E400010928A0402C01382128210938904009384
:104E50008804DF91CF911F910F910895A0E0B0E0F9
:104E6000E4E3F7E20C94C123EC01009721F4CB01B9
:104E70000E940126B8C0FC01E60FF71F9C012250DA
:104E80003109E217F30708F4ACC0D9010D911C9168
:104E9000119706171707B0F00530110508F49FC0E9
:104EA000C80104978617970708F499C002501109A2
:104EB000061B170B019311936D937C93CF010E94F6
:104EC00096268DC05B01A01AB10A4C01800E911E7E
:104ED000A0918A04B0918B0440E050E0E12CF12CC9
:104EE000109709F44AC0A815B905D1F56D907C90CA
:104EF0001197630182E0C80ED11CCA14DB0480F153
:104F0000A3014A195B096A0182E0C80ED11C1296FE
:104F1000BC9012971396AC91B5E0CB16D10440F03B
:104F2000B282A38351834083D9016D937C930AC0DD
:104F30000E5F1F4FC301800F911FF9019183808382
:104F4000EB2DFA2FE114F10431F0D7011396FC9305
:104F5000EE93129744C0F0938B04E0938A043FC011
:104F60008D919C9111974817590708F4AC017D0168
:104F700012960D90BC91A02DB3CF80918804909192
:104F8000890488159905E1F446175707C8F48091FC
:104F9000280190912901009741F48DB79EB7409167
:104FA0002C0150912D01841B950BE817F907C8F4CB
:104FB000F0938904E0938804F901718360830FC042
:104FC000CB010E9401267C01009759F0A801BE0187
:104FD0000E94FD27CE010E949626C70104C0CE0183
:104FE00002C080E090E0CDB7DEB7EEE00C94DD23A8
:104FF00081E090E0F8940C940628FB01DC0102C0EB
:1050000001900D9241505040D8F7089510E0C4EE41
:10501000D0E004C0FE010E9411252196C53ED107B3
:06502000C9F7F894FFCF70
:105026000F00F401D0070400040000803FFFFFFFDB
:10503600FF00E100000000000001C10FC10FC10F19
:10504600C10FC10F0100000000008C0480000400A5
:105056000F0020003700550078009C01B501CF01F4
:10506600EA0107022602470269028E02B502DE0243
:105076000A0300C18081000000018001800180FFD9
:105086007FFF7FFF7F00000000100B7D0AA80A57F4
:105096000BD90AB70ACB0A00000000830BD60B0C0B
:1050A60010990B6A0F34101010000000009D016D5E
:1050B60001CD01410165015101420100000000E7F7
:1050C6001000000000741100000000190A00000022
:1050D600007411426C7565746F6F746876657262E0
:1050E600696E64756E672068657267657374656C52
:1050F6006C74004665686C6572204472656862650A
:10510600776567756E677373656E736F7273004646
:1051160065686C65722042657363686C65756E6957
:1051260067756E677373656E736F7273000D0A0031
:2070000055C000006EC000006CC000006AC0000068C0000066C0000064C0000062C0000043
:2070200060C000005EC00000F2C400005AC0000058C0000056C0000054C0000052C00000EE
:2070400050C0000078C000004CC000004AC0000048C0000046C0000044C0000042C00000BE
:2070600040C000003EC000003CC000003AC0000038C0000036C0000034C0000032C0000048
:2070800030C000002EC000002CC000002AC0000028C0000026C0000024C0000022C00000A8
:2070A00020C000001EC000001CC0000011241FBECFEFDAE0DEBFCDBF11E0A0E0B1E0E2E3BC
:2070C000FFE702C005900D92A83AB107D9F711E0A8EAB1E001C01D92AE3BB107E1F78FD30B
:2070E00026C78ECFF89410926F0010928100109285001092840081E085BF15BE47985D9AEB
:20710000289A0C94000008952091B2013091B3012F5F3F4F3093B3012093B201932F37FFA6
:2071200003C08EEF831B982F990F921710F447980895479A08951F920F920FB60F9211246E
:207140002F938F939F93EF93FF9310928500109284008091A8019091A901009741F00197D3
:207160009093A9018093A801892B09F45D9A8091AA019091AB01009741F001979093AB0126
:207180008093AA01892B09F4289AE0E0F0E0859194918F5F9F4F49F08091AC019091AD0151
:2071A00001969093AD018093AC01FF91EF919F918F912F910F900FBE0F901F90189584E0BC
:2071C0008093E9000DC08091E8008B778093E80003C08EB3882351F08091E80082FFF9CFBE
:2071E0008091E80085FFEFCF8091F1000895982F83E08093E9008091E80085FD0DC0809136
:20720000E8008E778093E80003C08EB3882369F08091E80080FFF9CF9093F1005D9884E6CB
:2072200090E09093A9018093A80108954F925F926F927F928F929F92AF92BF92CF92DF921E
:20724000EF92FF920F931F93CF93DF9384E08093E9008091E80082FF57C2289884E690E067
:207260009093AB018093AA01AADF182F853481F48CE49DE19093AD018093AC0107B600FC4B
:20728000FDCFF999FECF81E180935700E89503C0843519F494DF8DE00DC28C34E1F38035F9
:2072A000D1F3843721F484E4A2DF80E003C2813611F489E5FFC18134B1F481DF182F7FDFE3
:2072C00090E0880F991FAA2797FDA095BA2F312F330F20E0442737FD4095542F822B932B68
:2072E000A42BB52BB8C1803711F483E5E3C1833549F4C0E0D1E089917ADF21E0C730D20714
:20730000D1F7D9C1863521F481E371DF80E3D2C1833731F487E86BDF85E969DF8EE1CAC149
:207320008536B9F4E0E0F0E093E085E090935700E89507B600FCFDCF80935700E89507B65D
:2073400000FCFDCFE058FF4FA0E7E030FA0771F7A2CF823739F4E1E0F0E089E08093570024
:207360008491A8C1863439F4E0E0F0E089E08093570084919FC18E3439F4E3E0F0E089E0E5
:2073800080935700849196C1813539F4E2E0F0E089E08093570084918DC1823631F489E521
:2073A00026DF80E024DF80E885C1823419F0873609F0E5C01092AD011092AC0100DF082FE8
:2073C000FEDEF82EFCDE682E8554823008F071C1902F80E0CF2DD0E0C82BD92B10926F00B3
:2073E000173609F04BC081E180935700E895DD24CC24C3943FC0E090AE01F090AF010091CC
:20740000B0011091B101B6E46B16D9F4ED2DF0E0EE29FF29E4918E2FEADEDD2081F082E08D
:2074200090E0A0E0B0E0E80EF91E0A1F1B1FE092AE01F092AF010093B0011093B101DC2470
:2074400018C0D801C701B695A7959795879559D5CEDE82E090E0A0E0B0E0E80EF91E0A1FF2
:207460001B1FE092AE01F092AF010093B0011093B1012197209709F0BECF7DC08090AE01F5
:207480009090AF01A090B001B090B10196E4691609F05DC083E0F40180935700E89507B63E
:2074A00000FCFDCF54C0F6E46F1661F5772031F1E090AE01F090AF010091B0011091B1019E
:2074C0007EDED82ECC24852D90E08C299D29F7010C0140925700E895112482E090E0A0E08B
:2074E000B0E0E80EF91E0A1F1B1FE092AE01F092AF010093B0011093B10102C060DE582E1A
:20750000742423C0E090AE01F090AF010091B0011091B10116950795F794E79450DE682FFA
:20752000C701F7D48091AE019091AF01A091B001B091B1010296A11DB11D8093AE01909349
:20754000AF01A093B001B093B101219704C05524772444244394209709F0A5CF96E46916B6
:2075600041F485E0F40180935700E89507B600FCFDCF8DE03CDE82E080936F009CC0833492
:2075800071F40091AE011091AF0119DE90E021E0F8010C0120935700E89511247CCE8336C8
:2075A00019F5E090AE01F090AF010091B0011091B10105DEF701E16090E021E00C0120938C
:2075C0005700E895112482E090E0A0E0B0E0E80EF91E0A1F1B1FE092AE01F092AF0100936A
:2075E000B0011093B10157CE8D3661F4E091AE01F091AF0185E080935700E89507B600FCF2
:20760000FDCF49CE823551F4E091AE01F091AF0105911491812FEBDD802F4CC0843421F5FE
:20762000E090AE01F090AF010091B0011091B10116950795F794E794C2DD682FC70169D4DE
:207640008091AE019091AF01A091B001B091B1010296A11DB11D8093AE019093AF01A093D8
:20766000B001B093B10117CE843609F5E090AE01F090AF010091B0011091B101D801C70142
:20768000B695A795979587953CD4B1DD82E090E0A0E0B0E0E80EF91E0A1F1B1FE092AE010A
:2076A000F092AF010093B0011093B10104C08B3111F08FE39CDD83E08093E9009091E8002B
:2076C0008091E8008E778093E80095FF04C010C08EB38823C9F08091E80080FFF9CF809193
:2076E000E8008E778093E80003C08EB3882361F08091E80080FFF9CF84E08093E9008091F1
:20770000E8008B778093E800DF91CF911F910F91FF90EF90DF90CF90BF90AF909F908F90AC
:207720007F906F905F904F9008959091B601892F8F77813249F58091B7018032A1F081328A
:2077400019F5913A09F58091E800877F8093E8008DE091E067E070E00BD28091E8008B770B
:207760008093E8000895913279F48091E800877F8093E8008DE091E067E070E05DD2809192
:20778000E8008E778093E800089582E061EC42E0B5D083E061E842E1B1D084E060E842E1EF
:2077A000ADC084B7877F84BF88E10FB6F89480936000109260000FBE20E880E090E00FB63F
:2077C000F89420936100809361000FBE81E085BF92E095BF3F9A209A559AE1E6F0E02083A1
:2077E000108247985D9A289A109289008AEF8093880090936F0083E080938100F0C0409116
:20780000000850910108109201081092000894B714BE88E10FB6F8948093600010926000D5
:207820000FBE292F30E0F901E270F07091FD18C090FF05C0859194918F5F9F4F81F423FFFF
:207840000FC08091090190910A014817590741F0E0E0F0E0859194918F5F9F4F09F042DC64
:20786000A0DF78941092AD011092AC010CC0DEDC36D38091AC019091AD0181549F4110F00D
:207880001092140141DC80911401882381F78091E00081608093E00025DC80E090E0089598
:2078A000FA01923049F0933061F09130F9F485E191E022E130E01EC087E291E02EE330E04D
:2078C00019C0882329F485E691E024E030E012C0813029F489E691E022E230E00BC0823006
:2078E00029F48DE891E028E130E004C080E090E020E030E091838083C90108958093E9004E
:207900008091EB0081608093EB001092ED006093EC004093ED008091EE00881F8827881F62
:2079200008958091B60188238CF403C08EB38823B1F08091E80082FFF9CF8091E8008B772A
:207940008093E80008958EB3882349F08091E80080FFF9CF8091E8008E778093E800089594
:20796000EF92FF920F931F9345D04CD008ED10E0F80180818F77808380818068808380819B
:207980008F7D808319BC1EBA1092B40180EEE82EF12CF70180818B7F8083F8018081816052
:2079A000808380E060E042E0A9DFE1EEF0E080818E7F8083E2EEF0E0808181608083808144
:2079C00088608083F70180818E7F8083F8018081806180831F910F91FF90EF900895E7ED06
:2079E000F0E08081816080838AE482BF81E08093B501B6CFE8EDF0E080818E7F808310921C
:207A0000E20008951092DA001092E10008951F920F920FB60F9211242F933F934F935F93F6
:207A20006F937F938F939F93AF93BF93EF93FF938091DA0080FF1BC08091D80080FF17C0B2
:207A40008091DA008E7F8093DA008091D90080FF0BC080E189BD82E189BD09B400FEFDCF36
:207A600081E08EBB3BD203C019BC1EBA37D28091E10080FF17C08091E20080FF13C0809138
:207A8000E2008E7F8093E2008091E20080618093E2008091D80080628093D80019BC85E049
:207AA0008EBB1CD28091E10084FF2CC08091E20084FF28C080E189BD82E189BD09B400FEC5
:207AC000FDCF8091D8008F7D8093D8008091E1008F7E8093E1008091E2008F7E8093E20012
:207AE0008091E20081608093E2008091B401882331F48091E30087FD02C081E001C084E067
:207B00008EBBECD18091E10083FF21C08091E20083FF1DC08091E100877F8093E10082E06A
:207B20008EBB1092B4018091E1008E7F8093E1008091E2008E7F8093E2008091E2008061E9
:207B40008093E20080E060E042E0D8DEC7D1FF91EF91BF91AF919F918F917F916F915F9130
:207B60004F913F912F910F900FBE0F901F9018959C014091BC015091BD014617570718F49D
:207B8000F90190E044C06115710511F0AB01F8CF8091E8008E778093E80040E050E0F0CF0F
:207BA0008EB3882309F444C0853009F443C08091E80083FF02C081E008958091E80082FD70
:207BC00031C08091E80080FF22C08091F3009091F200782F60E0292F30E0262B372B07C07A
:207BE00081918093F100415050402F5F3F4F4115510519F02830310598F390E02830310566
:207C000009F491E08091E8008E778093E8004115510531F6992321F605C08EB3882341F075
:207C2000853041F08091E80082FFF7CF80E0089582E0089583E008959C016115710529F47C
:207C40008091E8008B778093E800F90126C08EB3882391F1853091F18091E80083FF02C06C
:207C600081E008958091E80082FFF1CF06C08091F10081936150704059F02091F300809191
:207C8000F200322F20E090E0822B932B892B79F78091E8008B778093E80061157105B9F601
:207CA00005C08EB3882341F0853041F08091E80080FFF7CF80E0089582E0089583E00895C2
:207CC0000F931F93DF93CF9300D0CDB7DEB7E6EBF1E08091F100819381E0EE3BF807C9F792
:207CE00024DD8091E80083FFE4C08091B6019091B701953009F46DC0963040F4913081F1A7
:207D0000913070F0933009F0D4C02AC0983009F4A3C0993009F4B2C0963009F0CAC07CC023
:207D2000803809F4C6C0823809F0C3C08091BA0187708093E9008091EB001092E9002091DB
:207D4000E800277F2093E80090E025E0969587952A95E1F781708093F1001092F10087C0D8
:207D6000882319F0823009F0A4C08F71823009F0A0C08091B801882331F52091BA01277097
:207D800009F497C02093E9008091EB0080FF1BC0933021F48091EB00806213C08091EB0018
:207DA00080618093EB0081E090E002C0880F991F2A95E2F78093EA001092EA008091EB00E5
:207DC00088608093EB001092E9008091E800877F51C0882309F06DC01091B8011F770FB79B
:207DE000F8948091E800877F8093E8009ADD8091E80080FFFCCF8091E3008078812B809398
:207E0000E30080688093E300112311F482E001C083E08EBB0FBF4DC08058823008F049C033
:207E20008091B8019091B9016091BA01AE014F5F5F4F36DDBC01009709F43BC08091E8008E
:207E4000877F8093E80089819A8192DE8091E8008B778093E8002DC0803859F58091E800AA
:207E6000877F8093E8008091B4018093F1008091E8008E778093E80054DD1BC08823C9F4CA
:207E80009091B8019230A8F48091E800877F8093E8009093B40145DD8091B401882331F420
:207EA0008091E30087FD02C081E001C084E08EBB6CDC8091E80083FF0AC08091EB0080624E
:207EC0008093EB008091E800877F8093E8000F900F90CF91DF911F910F91089508951F9360
:207EE0008EB3882361F01091E9001092E9008091E80083FF01C0E4DE17701093E9001F916F
:207F00000895F999FECF92BD81BDF89A992780B50895262FF999FECF1FBA92BD81BD20BDBD
:207F20000FB6F894FA9AF99A0FBE01960895F894FFCF4341544552494E4100777700080031
:207F40000000000000080112011001020000084123360001000201000109023E00020100FF
:207F600080320904000001020201000524001001042402040524060001070582030800FF0C
:207F800009040100020A000000070504021000010705830210000104030904220341007216
:207FA000006400750069006E006F0020004C0065006F006E006100720064006F0000001836
:1A7FC00003410072006400750069006E006F0020004C004C004300000000D7
:00000001FF
